:020000040000FA
:1000000010280000000000000000000000000000B8
:1000100000000000000000000000000000000000E0
:100020008316FF3085008601870104309F0083120C
:1000300040309F001F142830AD00B620AD0B1D28A6
:100040003030A5200F30A5200130A520B620B620E5
:100050000730A5208F30A5204330AE20B620573082
:10006000AE20B6202030AE20B6204430AE20B620E0
:100070006530AE20B6206330AE20B6206F30AE20A3
:10008000B6206430AE20B6206530AE20B620723087
:10009000AE20B6202030AE20B6202030AE20B620D4
:1000A000A401A501051D52280021051D522800218B
:1000B0000021A50A240CFE39A400051D6628A40A07
:1000C0000519602800210519602869282E30AE2006
:1000D0006B282D30AE202808A900B620A9030319EB
:1000E0007628051D6D280021051D57282808A90020
:1000F000B620A90303198128051D78280021051DB4
:100100005728250AF839031D9E2825080621860050
:10011000AE20A401A50100210519522800210519CE
:1001200052280021051952280021051952280021C2
:100130000519522820308600AE205228FF30860054
:10014000AE20A401A5015228A428860087018717A4
:1001500000008713B6200717871608008600203096
:10016000870087170000871307170800A630AC0028
:10017000AC0BB8281F15A530AC00AC0BBD281E0C6D
:080180007F390C3EA8000800C5
:100200002808A900B620290B0229080001308A001D
:100210002508073982070034132918291F292A299C
:100220003D296029003424080139820745345434BB
:10023000240803398207493441344E344D342408AC
:1002400007398207533455345234573444344B34CD
:1002500047344F3424080F39820748345634463423
:10026000FF344C34FF3450344A344234583443342D
:1002700059345A345134FF34FF3424081F3982076B
:1002800035343434FF343334FF34FF34FF34323404
:100290003D34FF347F34FF34FF34FF34FF343134D6
:1002A00036343D342F34FF34FF347E343C34FF3455
:1002B0003734FF34FF34FF343834FF3439343034CA
:1002C00024083F398207FF34FF34FF34FF34FF3402
:1002D0007F34FF34FF34FF34FF34FF34FF343F34C6
:1002E000FF34FF34FF34FF34FF34FF34FF34FF3476
:1002F0002E34FF34FF34FF34FF34FF34FF34FF3437
:10030000FF34FF34FF34FF34FF34FF34FF34FF3455
:10031000FF34FF34FF34FF34FF34FF34FF34FF3445
:10032000FF34FF34FF34FF34FF34FF342C34FF3408
:10033000FF34FF34FF34FF34FF34FF34FF34FF3425
:06034000FF34FF34FF341E
:02400E00793FF8
:00000001FF
